:1000000031C04BC037C349C048C047C046C045C0D7
:1000100044C043C042C041C040C03FC03EC00902CE
:10002000190001010080640904000001FF000000C4
:100030000705810308000A12011001000000088171
:10004000179F0C04010002000116035500530042E3
:1000500000740069006E00790053005000490004EC
:100060000309040011241FBECFE5D1E0DEBFCDBFE0
:1000700010E0A0E6B0E0E2EAF9E002C005900D92DF
:10008000A436B107D9F720E0A4E6B0E001C01D9284
:10009000AB3AB207E1F74CD482C4B2CFFC01DB012A
:1000A000AC014C5F5F4F619128E030E080E890E068
:1000B000762F782309F0C09A70916000072E00C057
:1000C0000000000000000A94D1F7C29A709160000D
:1000D000072E00C00000000000000A94D1F7990F1D
:1000E000B1999F5FC098C29886952150310901F758
:1000F0009D934E175F07B9F6089580916F00909118
:1001000070009C012F5F3F4F3093700020936F0071
:1001100020916C0027FF02C0880F991F80FD286086
:1001200020936800292F269520936900969587953E
:1001300080936A0064E670E088E690E0AFCFEF92CB
:10014000FF921F93CF93DF93162FEC017C01E60EF5
:10015000F11CCE15DF0529F0D0DF8091670089936F
:10016000F8CF812FDF91CF911F91FF90EF900895ED
:10017000DF92EF92FF920F931F93CF93DF93EC01E7
:100180007C01E60EF11C30E6D32ECE15DF0581F1A1
:10019000899180936B00B1DF809168008D258093F9
:1001A000680000E010E080916D0090916E000817EB
:1001B000190758F764E670E088E690E06FDF8091F9
:1001C000670090916B00891308C0909172008917A5
:1001D00021F0909171008913D8CF8091600090E058
:1001E00025E0880F991F2A95E1F7080F191FDBCF2B
:1001F00081E0DF91CF911F910F91FF90EF90DF9001
:100200000895CF93DF93FC018181811106C0F093A3
:100210009000E0938F0088E06BC0A481B0E0813053
:1002200041F48C918083F0939000E0938F0081E003
:100230005FC09281823011F49C9359C0492F47705E
:1002400021E030E001C0220F4A95EAF7833021F423
:1002500020958C91282304C0843021F48C91282B84
:100260002C9345C0853049F490936000B99887B3CA
:10027000856287BB88B3887D04C0863021F480E224
:1002800087BB88BB34C0873059F4EF01BF01CF0171
:10029000029604DFD0939000C0938F0084E028C0C2
:1002A000883031F4909372008381809371001FC075
:1002B000248135813093700020936F00893011F4D0
:1002C00080E211C08B3011F480EA0DC022813381AD
:1002D00030936E0020936D008A3011F480E403C0E7
:1002E0008C3029F480EC80936C008FEF01C080E0AB
:1002F000DF91CF910895DF92EF92FF920F931F93BA
:10030000CF93DF9308E010E0C0E0D0E8DD2EDC0EF4
:10031000D1BE9DD17C0184E3E81689E0F8060CF497
:10032000CD2DD6950150110989F78FEF8C0F81BF24
:100330000C2F10E00F5F1F4F81B790E008171907CF
:100340008CF085D18453994097FF03C09195819596
:1003500091098E159F0514F4C1B77C0181B78F5F99
:1003600081BFEACFC1BF61B780E090E0DF91CF915C
:100370001F910F91FF90EF90DF9003C3CF93C62F93
:100380002091800024FF0BC03091810028E82327B2
:1003900020938100FC01A2E8B0E08C2F04C02AE584
:1003A00020938000F7CF91919D938150E1F76C2FBE
:1003B00082E890E048D1CC5FC0938000CF9108954F
:1003C000CF93DF9360919100635067FDA4C080914B
:1003D0008E00CCE0D0E0C81BD109CB56DF4F809116
:1003E0008D008D3209F086C0683009F092C083EC30
:1003F000809375008AE58093620010927400888172
:10040000807631F0CE01FDDE8F3F09F462C068C016
:100410009A8110927E008981811106C010927F001E
:100420002EE730E082E050C0853019F490939200BE
:1004300048C0863081F58B81813041F487E390E0BC
:100440009093900080938F0082E121C0823041F42C
:100450008EE190E09093900080938F0089E117C027
:100460008330A1F4911108C08FE590E09093900043
:1004700080938F0084E00BC0923041F489E490E0D7
:100480009093900080938F0086E101C080E090E41B
:100490009093740025C0883069F0893019F49093E6
:1004A00094000FC08A3049F08B3059F48BE480936C
:1004B000810007C024E930E002C02EE730E081E08F
:1004C00003C02EE730E080E03093900020938F004F
:1004D00007C0988197FD8E8190E89093740007C0C3
:1004E0009F81911104C09E81981708F4892F8093F1
:1004F00061000FC08091740087FF0BC0CE0138DE11
:100500008F3F21F48EE18093620003C0811110922D
:100510006100109291008091620084FF55C080912B
:1005200061008F3F09F450C0C82F893008F0C8E03F
:100530008C1B809361009091750088E889278093D7
:100540007500CC2309F456C02091740027FF08C021
:100550006C2F86E790E0F3DDC82F893078F523C053
:1005600080918F009091900026FF0AC0A6E7B0E02E
:10057000FC012C2F34913D9331962150D9F708C0BE
:10058000DC01E6E7F0E02C2F3D9131932150E1F7BB
:100590002FEF2C0F30E02F5F3F4F820F931F909370
:1005A000900080938F006C2F86E790E04CD0CC5F5A
:1005B000CC3041F08FEF8093610004C08FEF8093C7
:1005C0006100CEE1C093620084E196B3987131F48A
:1005D0008150D9F71092920010928C00C1E08111E5
:1005E000C0E090917300C91759F0811184DEC09367
:1005F000730006C060E086E790E025D0C4E0DACF63
:10060000DF91CF910895AC9A8BB780628BBFE0E801
:10061000F0E08BE481838AE580830895A82FB92FC9
:1006200080E090E041E050EA609530E009C02D9113
:1006300082279795879510F084279527305EC8F319
:100640006F5FA8F30895EADF8D939D930895A6E068
:1006500088279927AA9569F00197E1F3B399FCCF10
:10066000B39BFECF81E09927A6B3019611F0A87144
:10067000D9F70895CF93CFB7CF93C395B39BE9F73D
:10068000B39B0BC0B39B09C0B39B07C0B39B05C012
:10069000B39B03C0B39B01C0D5C00F92DF93C09141
:1006A0008E00DD27CB56DF4F012EB39B03C0DF91B9
:1006B0000F90E6CF2F930F931F934F932FEF4F6F12
:1006C00006B303FB20F95F933F9350E03BE065C026
:1006D00016B30126502953FDC89556B3012703FBD5
:1006E00025F92F7306B3B1F05027102713FB26F915
:1006F00006B22230F0F000C016B3012703FB27F941
:100700000126502906B22430E8F54F77206816B349
:100710000000F6CF50274F7D206206B2102F000058
:1007200000C006B300265029102713FB26F906B295
:10073000E2CF4F7B06B3206400C0DACF01265029F8
:10074000187106B269F14E7F2160012F16B328C0DF
:10075000002650294D7F06B22260102F29C00126A5
:1007600050294B7F06B22460012F2DC016B30126FD
:100770005029477F2860000006B22EC04F7E06B386
:10078000206130C0422706B3499300265029102724
:1007900006B24FEF13FB20F9297F16B379F21871D7
:1007A00059F10126502906B2012703FB21F9237FC5
:1007B00006B371F2002650293150D0F006B210274E
:1007C00013FB22F9277E16B351F201265029012787
:1007D00003FB06B223F92F7C49F2000006B3102771
:1007E00013FB24F90026502906B22F7939F270CF75
:1007F00010E21ABF002719C03B503195C31BD040EF
:1008000010E21ABF0881033C09F10B34F9F0209182
:100810008C001981110F1213EDCF4A81441F093644
:1008200051F10D3211F0013E29F7009393003F91F1
:100830005F914F911F910F912F91DF910F90CAB748
:10084000C5FD1BCFCF91CFBFCF91189520919300BD
:10085000222369F310919100112379F534307AF154
:100860003093910020938D0010918E003BE0311B5E
:1008700030938E0024C0009191000130F4F40AE519
:100880004F7049F43091620034FD1AC00093620049
:10089000C5E7D0E019C03091800034FD11C000934D
:1008A0008000C1E8D0E010C0052710E000C021C0E2
:1008B000052710E0C89508BB14C03AE501C032ED29
:1008C000032EC0E0D0E032E017B31861C39A08B33A
:1008D00017BB58E120E84FEF20FF052708BB2795FD
:1008E00017951C3F28F700004552B0F720FF052759
:1008F000279508BB17951C3FB8F629913A9561F7E3
:10090000077E10919200110F08BBC250D04011F029
:1009100010938C0010E21ABF086017B3177E402FA7
:10092000477E54E05A95F1F708BB17BB48BB7FCF11
:1009300080E287BB88BB80E090E01BD08F3F09F04E
:1009400081BFBB9A84E1E2EBF1EF3197F1F700C090
:1009500000008150C1F7BB989EE088E10FB6F89483
:10096000A89581BD0FBE91BD4EDE7894A89528DD77
:10097000FDCFE199FECF1FBA8EBBE09A99278DB3C8
:100980000895262FE199FECF1CBA1FBA8EBB2DBB4E
:100990000FB6F894E29AE19A0FBE01960895F89482
:0209A000FFCF87
:0409A20032FF5A00C6
:00000001FF
